:020000040800F2
:104000000845002099420008D967000801530008BC
:10401000AD590008494B00087985000800000000F0
:10402000000000000000000000000000AD4100089A
:104030003F4E00080000000035420008854200089D
:10404000B3420008B3420008B3420008B34200087C
:10405000B3420008B3420008B3420008B34200086C
:10406000B3420008B3420008B3420008B34200085C
:10407000B14C0008B3420008B34C0008B34200083A
:10408000B3420008B3420008B3420008B34200083C
:10409000B3420008B3420008B3420008B34200082C
:1040A000B3420008B3420008B3420008B34200081C
:1040B000ED7B00080B7C00080D7C0008B342000873
:1040C000B3420008B3420008B3420008B3420008FC
:1040D000B34200088D7E0008D17E0008D57E00081E
:1040E000834E0008B3420008B3420008B342000800
:1040F000B3420008B3420008B3420008B3420008CC
:10410000B3420008B3420008B3420008B3420008BB
:10411000B3420008B3420008B3420008B3420008AB
:10412000B3420008B3420008B3420008B34200089B
:10413000DFF80CD000F028FA004800470190000892
:104140000845002080F309887047EFF30980704725
:10415000684680F3098804480078C00714BF02202D
:10416000032080F3148870473C9D0008DFF818C0D6
:10417000EFF305831B0618BF6047EFF31483DB07DB
:1041800008BF604700DF7047ED900008DFF818C0F7
:10419000EFF305831B0618BF6047EFF31483DB07BB
:1041A00008BF604700DF704795920008EFF3098071
:1041B000816911F8021C39BB90E80F10E047EFF35A
:1041C000098C194B93E80600914218D059B10CB4F0
:1041D0004FF0010381F826302CE9F00FC1F82CC014
:1041E00005F072FA0CBC1A60D2F82CC0BCE8F00FD3
:1041F00092F826308CF309881BB192F82500CCF890
:1042000000006FF0020E704710B5084A1268914224
:1042100009D8074C54F8214090E80F10A047EFF35D
:10422000098C8CE80F0010BDE40000201447000842
:104230001447000805F016F9114B93E80600914267
:104240001BD00CB44FF0000381F82630EFF3098C3B
:104250002CE9F00FC1F82CC005F036FA0CBC1A603E
:10426000D2F82CC0BCE8F00F8CF3098892F8263005
:104270001BB192F82530CCF800306FF0020E704779
:10428000E400002005F0F0FAD6E7000004F02CFF6F
:1042900005F0EAFAD0E700000648804706480047E4
:1042A000FEE7FEE7FEE7FEE7FEE7FEE7FEE7FEE7E6
:1042B000FEE7FEE76D7B00083141000840EA01039C
:1042C0009B0703D009E008C9121F08C0042AFAD2CC
:1042D00003E011F8013B00F8013B521EF9D2704790
:1042E000D2B201E000F8012B491EFBD27047002238
:1042F000F6E710B513460A4604461946FFF7F0FFE5
:10430000204610BD30B505462A460B4612F8010B73
:1043100013F8014B08B1A042F8D01CB1002802D01C
:104320006D1CF1E7284630BD10B5044604E00B785B
:1043300000F8013B03B1491C521EF8D2204610BDC3
:10434000421C10F8011B0029FBD1801A704710B5E0
:10435000002200E0521C835C8C5CA34201D1002B44
:10436000F8D1D8B2E1B2401A10BD30B504460020F1
:10437000034600E05B1C934203D2E05CCD5C401B33
:10438000F8D030BD034611F8012B00F8012B002AAC
:10439000F9D11846704770B5064604F0BBF90468B9
:1043A00005460A220021304600F06DF82C6070BDF1
:1043B00070B5064604F0AEF9046805460A220021ED
:1043C000304600F098F82C6070BD2DE9F05F05468E
:1043D000002092469B4688460646814640241BE0C4
:1043E000284641464746224600F02FF853465A4693
:1043F000C01A914110D311461846224600F016F813
:104400002D1A67EB01084F4622460120002100F0DB
:104410000DF817EB00094E41201EA4F10104DFDC6A
:10442000484631462A464346BDE8F09F202A04DB31
:10443000203A00FA02F1002070479140C2F12003B7
:1044400020FA03F3194390407047202A04DB203AF6
:1044500021FA02F00021704721FA02F3D040C2F1A4
:10446000200291400843194670473A2800D230385C
:1044700020F02002412A01D3A2F13700884201D363
:104480004FF0FF3070472DE9F04791460F468046C8
:104490000446002614F8015B2DB100F087F800688F
:1044A000405DC007F6D12B2D02D02D2D18D0641EF3
:1044B0004A463946204600F07DF827B13968A142C6
:1044C00001D1C7F8008071054FF002040BD54042BE
:1044D000002803DD04F01EF90460A007BDE8F087A2
:1044E00046F48066E4E70028F8DA04F013F9046083
:1044F0006FF00040F2E72DE9F04791460E46804606
:104500000446002514F8017B2FB100F04FF8006835
:10451000C05DC007F6D12B2F02D02D2F1ED0641EF8
:104520004A463146204600F094F826B13268A2424D
:1045300001D1C6F800806A054FF0020418D50023A7
:10454000D0EB030563EB01025D1B934109DB002304
:10455000D0EB030063EB0101BDE8F08745F4806513
:10456000DEE704F0D7F8046000204FF00041F3E7E5
:10457000021E71F10002EFDA04F0CCF804604FF093
:10458000FF304108E8E70000064C074D06E0E06810
:1045900040F0010394E8070098471034AC42F6D38A
:1045A000FFF7CAFDA89E0008C89E00080048704793
:1045B000F49D00082DE9F05F82460078002715463B
:1045C0008B460AF10104B946302801D09DB113E0B1
:1045D00014F8010B0127782803D0582801D045B1E1
:1045E0000AE00DB1102D07D10027102514F8010B9A
:1045F00002E0082500E00A250026B0460EE005FB93
:10460000080005FB06F1012701EB10461FFA80F8B0
:10461000B6F5803F00D3B94614F8010B2946FFF7E1
:1046200024FF0028EBDABBF1000F05D00FB1641EA8
:1046300000E05446CBF80040B9F1000F06D004F07A
:1046400069F802210160C81EBDE8F09F48EA0640F3
:10465000FAE72DE9F74F4FF00009009C1546CA46CE
:1046600014F8010B302801D0ADB115E014F8010B9E
:104670004FF00109782803D0582801D04DB10BE044
:104680000DB1102D08D14FF00009102514F8010BC1
:1046900002E0082500E00A2500273E46B8464FEA1A
:1046A000E57B16E0A5FB07230BFB073105FB0800A4
:1046B00005FB0616030CD71846F100061FFA80F812
:1046C000381E4FF0010976F5803000D3CA4614F841
:1046D000010B2946FFF7C9FE0028E3DA019838B13B
:1046E000B9F1000F01D0641E00E0009C0198046045
:1046F000BAF1000F08D004F00DF802210160C81EC5
:10470000014603B0BDE8F08F310441EA174148EAA1
:104710000740F6E70000000010B58EB02BA1012085
:1047200003F000FA00F072F810212D4800F0A9FD06
:104730000020ADF820004FF48271ADF82210ADF8E2
:1047400024000221ADF826100121ADF828104902FD
:10475000ADF82A100821ADF82C10ADF82E00072076
:10476000204CADF8300008A9204603F000F90121E3
:10477000204602F0A7FF4FF47A7000F079FB03F0B7
:104780000FF8194C024619A16060684603F0AEFFAD
:104790006946012003F0C6F9184AD4F80410002035
:1047A00052F820308B420ED10F49083151F82020A9
:1047B00013A1684603F09AFF6946012003F0B2F99D
:1047C0000EB0012010BD401CEAE7000073466C618A
:1047D000736820496E69742E2E2E0D0A00000000A9
:1047E0000008014000300140C40000204678462007
:1047F00049643D253034780D0A000000549D0008BE
:104800004578463D25730D0A0000000038B50121AA
:10481000042002F059FD0121080302F055FD20207B
:10482000ADF8000003208DF802001820104C8DF820
:1048300003006946204600F09DFC8020ADF8000092
:104840006946204600F096FC4020ADF800000420A8
:104850008DF803006946204600F08CFC1021ADF86D
:1048600000108DF803106946204600F083FC38BD27
:1048700000080140F0B50E4689B004465EA101F083
:1048800051FC624D18B10220687109B0F0BD142EC0
:10489000FBD35FA1204601F045FC0128F5D1E07B68
:1048A00000263038C7B2EE8304F11100FFF773FD24
:1048B00081B2481E40F20B429042E6D20A2901D250
:1048C000143409E0642901D2153405E0B1F57A7F8A
:1048D00001D2163400E01734012FD6D1204600F063
:1048E00049F9020004D54EA101A803F0FFFE23E020
:1048F000B2F5024F0AD0A0F50942293A21D0072A81
:10490000C3D104F10C0004F07DF9BEE74AA10120F7
:1049100003F008F9608940BA2883207B0028B4D1CD
:104920004848627B0271A37B4371E17B81710091F6
:1049300045A101A803F0DAFE01A9012003F0F2F875
:10494000A3E749A1012003F0EDF8608940BA28836C
:1049500004F10C0002F072FDA07CC0EB001080009E
:10496000A8840CD043A1012003F0DCF8AA8C45A157
:1049700001A803F0BBFE01A9012003F0D3F8E07CFD
:10498000012820D1A08A47BAEFB141484289BA42F2
:1049900019D2A88A052816D23B463EA101A803F0E9
:1049A000A5FE01A9012003F0BDF840A1012003F0FC
:1049B000B9F84248012107810170002001F042F856
:1049C0000620287061E7AE823D4AE08A218B92F88A
:1049D000233040BA49BA834201D0052805D292F863
:1049E00022308B4291D005298FD382F8230082F8A0
:1049F000221002F0F3FF48E72B51495552433A2069
:104A000022636C6F736564222C30000088260020BE
:104A10002B51495552433A202272656376222C006D
:104A2000436865636B5061636B6574204572723DCA
:104A300025640D0A000000003C3C5B383030315DDD
:104A40000D0A0000AE2F002049456E3D253032583A
:104A50002043456E3D253032582052456E3D25306D
:104A600032580D0A000000003C3C5B383932395D99
:104A70000D0A0000556E617574686F72697A65641D
:104A8000210D0A005543743D25640D0A0000000005
:104A9000220C00204375725665723D2564204E65D8
:104AA000775665723D25640D0A00000055706772E7
:104AB000616465206E6F77210D0A00005C2B002079
:104AC000320D002070B51E4E002500BFC5EBC5009D
:104AD00000EB0510315C69B38419A078062829D24F
:104AE000DFE800F028280312281F04F10F01042238
:104AF000362004F0ADF90320A070DFF848C000DFD5
:104B0000C830C4F8130015E0DFF838C000DFD4F86F
:104B1000131088420ED920461721FFF7E8FB00202A
:104B200007E0DFF820C000DFD4F81310884201D975
:104B30000620A0706D1C15F0FF05C7D070BD0000E9
:104B400085300020A99800080348026803480188BE
:104B500003A003F0A7FDFEE7440000203C00002076
:104B60000D0A5B4246485D463D25642C4C3D256C54
:104B70007500000030B50446002501F0E8FF00286C
:104B800001DA681E30BD0021421E02E0635C5D4018
:104B9000491C9142FADB204410F8010CA84202D0D3
:104BA0006FF0010030BD0A4900200A18231892F85E
:104BB000B6201B799A4203D1401C0628F5DB04E09D
:104BC000062802DA6FF0020030BD208840BA30BDFE
:104BD000220C002070B5134D134E044601280FD04F
:104BE000022C1DD111A1002002F09CFF2C70DFF8D7
:104BF0005CC0306800DFBDE87040022003F050BAAE
:104C000013A1002002F08EFF2C70DFF840C0306846
:104C100000DF012003F044FA14494FF4807008606B
:104C200070BD00001800002054000020446562752B
:104C30006720434F4D2073656C63657420746F204B
:104C40004D6F64656D210D0A000000008599000814
:104C5000446562756720434F4D2073656C636574CE
:104C600020746F20475053210D0A000010080140A6
:104C700010B507A1012002F055FF0B480BA100F170
:104C8000E602B0F80E31BDE81040012001F0ACB8EA
:104C9000436F6E6E656374417574685365727665B3
:104CA000723E3E0D0A000000220C002055445000C8
:104CB000704703F0F3B80000C10002D50249086054
:104CC00070470249486070470404024000000240F7
:104CD000C10002D502490860704702494860704728
:104CE00004040240000002400029016802D041F0A3
:104CF000010102E04FF6FE721140016070470000B2
:104D000001684FF6FE7211400160002101604160B0
:104D10008160C1603149314A0839904203D1486805
:104D200040F00F0006E02D4A1432904204D148684A
:104D300040F0F00048607047284A2832904203D182
:104D4000486840F47060F5E7244A3C32904203D151
:104D5000486840F47040EDE7204A5032904203D159
:104D6000486840F47020E5E71C4A6432904203D161
:104D7000486840F47000DDE7184A7832904203D169
:104D8000486840F07060D5E7154A111F904203D182
:104D9000086840F00F0006E0114A1432904204D136
:104DA000086840F0F000086070470D4A28329042D1
:104DB00003D1086840F47060F5E7094A3C3290423C
:104DC00003D1086840F47040EDE7054A5032904244
:104DD000EAD1086840F47020E5E7000008000240CE
:104DE0000804024001460020CA0001D5034A00E041
:104DF000034A12680A4200D00120704700040240B2
:104E00000000024030B5036847F6F07293430C6A25
:104E10008A682243D1E904452C4322438C6922430A
:104E2000CC6922434C6A22438C6A22431A430260B3
:104E3000CA6842600A6882604968C16030BD7047D4
:104E4000F0B5521E13D464235FF00A04B0FBF3F5EF
:104E500003FB150595FBF4F695FBF4F7B0FBF3F0B7
:104E600004FB175566F31F158D54521EEED5F0BD89
:104E700003E00521491E89B2FCD2401E80B2F8D25F
:104E80007047704738B50121042002F01DFA022452
:104E9000ADF8004010208DF8030003208DF80200CB
:104EA0006946124800F066F910481030046000BFEF
:104EB00000BF00BF00BF00BF00BF00BF00BF0B4965
:104EC00014310C6000BF00BF00BF00BF00BF00BFB7
:104ED00000BF00BF046000BF00BF00BF00BF00BF35
:104EE00000BF00BF00BF0C6038BD000000080140DB
:104EF00070B505464FF43026304600F059F80428C6
:104F000011D1094C206940F00200206165612069DF
:104F100040F040002061304600F04AF8216941F637
:104F2000FD721140216170BD00200240084904203B
:104F3000CA68D20701D001207047CA68520701D55C
:104F400002207047C968C906FBD5032070470000DE
:104F5000002002400248016941F080010161704770
:104F600000200240F0B506464FF400570D46384683
:104F700000F01EF804280CD1064C206940F0010016
:104F800020613580384600F013F82169BA1E1140BF
:104F90002161F0BD002002400348024941600349FD
:104FA000416070472301674500200240AB89EFCD87
:104FB00000B50346FFF7BAFF03E000BFFFF7B6FFF7
:104FC0005B1E012803D0002B00D1052000BD002B63
:104FD000F4D1FAE72DE9F041DFF818C100DF4649C6
:104FE0004A694B78821A012B7ED00023642A22D989
:104FF00048614248007800287AD14149414D4FF438
:105000007A76C879A8B3088C401C80B20884B0F5C1
:10501000967F2FD90B843CA1012002F083FDDFF89D
:1050200000C1286800DF3FA000F0C4FF3046DFF871
:1050300000C100DF5AE03F4C8878322A0FD20028A6
:1050400056D1012088700DE0012200E000220221EB
:10505000204600F018F9BDE8F04100F091B90128B0
:1050600046D18B700221204600F002F90028EDD1D4
:10507000EAE7FFE7304C608C401C80B26084B428C3
:1050800008D92EA1012002F04DFDDFF894C0286858
:1050900000DF2BE0DFF8B8C000DFE08B4FF6FF71D8
:1050A000884201D2401CE0832A4FB889884201D24D
:1050B000401CB881DFF8A0C000DFE18B4FF46160D5
:1050C000814215D9B989814212D924A1012002F067
:1050D00029FDDFF84CC0286800DF12A000F06AFF4D
:1050E0003046DFF84CC000E002E000DF02F068FD6F
:1050F000BDE8F081A99800083800002018000020C1
:10510000AE2F00205400002055617274315278494E
:1051100064656C54696D656F7574210D0A0000003B
:105120008599000841542B51504F57440D0A0000F7
:105130004192000800080140882600204D6F6465F8
:105140006D5561727454696D656F7574210D0A0037
:10515000F19A00089E2F0020519B0008536572763B
:1051600065724F66666C696E6554696D656F7574BE
:10517000210D0A00F0B5CA78002502F00F03D2060F
:1051800001D58A7813430A784FF00F0E12F0FF0F03
:105190004FF001021CD004680F8802FA05F6374070
:1051A000B74211D14FEA850C0EFA0CF724EA070733
:1051B00003FA0CF43C43CF78282F02D0482F02D0BA
:1051C00002E0466100E006616D1C082DE4D3046036
:1051D0000C88FF2C1ED944685FF0000606F1080712
:1051E00002FA07F50F882F40AF420FD14FEA860C25
:1051F0000EFA0CF7BC4303FA0CF73C43CF78282F88
:1052000000D14561CF78482F00D10561761C082E6A
:10521000E4D34460F0BD0000F0B5144C002801DA7E
:10522000E36900E06368420D120185B2C0F30157E3
:105230009540C0F30346032F05D0C2020AD50322CE
:10524000B240934307E023F07062636823F0706319
:10525000636002E0AB4343F0706201B12A4300286F
:1052600001DAE261F0BD6260F0BD000000000140C3
:1052700002460020D2680A4200D0012070474161F6
:105280007047016170470AB1016170474161704721
:10529000F0B503460025007887B016462C462F4609
:1052A000E0B10A786846CAB107E0C2557F1C3D2AC2
:1052B00014D03B2A12D0491C641C0A780AB1142C61
:1052C000F3DB3D210155641C0027075501461846B4
:1052D000FFF718F8002802D0204407E0002007B0AC
:1052E000F0BD00BF401C06F8011B6D1C0178202991
:1052F00003D93B2901D0282DF4DB37702846EEE78F
:10530000034802680348018803A003F0CBF9FEE7D5
:10531000440000203C0000200D0A5B4846485D46E2
:105320003D25642C4C3D256C750000000F4810B5E0
:10533000416A41F001014162416A4908C907FBD055
:105340007D2002F027F808B101F0CAFF45F2555060
:1053500000F02AF8062000F01BF84FF4FA7000F075
:105360001DF8BDE8104000F003B800000010024036
:1053700002494CF6CC400860704700000030004005
:1053800002494AF6AA200860704700000030004039
:1053900001494860704700000030004001498860C2
:1053A000704700000030004001490860704700006D
:1053B0000030004038B501211C2001F085FF10208D
:1053C0008DF8030003208DF802004FF40050334C99
:1053D000ADF8000069462046FFF7CCFEA015304D21
:1053E000ADF8000069462846FFF7C4FE6015ADF829
:1053F000000069462846FFF7BDFE4FF48040ADF837
:10540000000069462046FFF7B5FE0023184600F06D
:105410004DF85B1C022BF9DB224D02212846FFF7D9
:1054200027FFA0B3002202212846FFF72CFFFFF739
:10543000A7FF0024204600F053F81E20DFF868C0C4
:1054400000DF02212846FFF713FF18B300220221D4
:105450002846FFF718FFFFF793FF641C022CE9DBD7
:1054600002212846FFF704FFB0B10022022128469E
:10547000FFF709FFFFF784FF0023184600F016F836
:105480005B1C022BF9DB012000F044F838BDFFE77C
:105490000122C8E70122DAE70122E7E70010014014
:1054A000000C014000080140419200080A4940B147
:1054B0000A4A012808D0022809D04FF480404861E8
:1054C00070474FF40050FAE74FF4807001E04FF45A
:1054D000007010607047000000100140140C014083
:1054E0000A4940B10A4A012808D0022809D04FF4DD
:1054F0008040086170474FF40050FAE74FF4807025
:1055000001E04FF40070106070470000001001408F
:10551000100C01402DE9F04F2F4D05F10C06B71C82
:1055200005F10808002405F10A0905F1060A88B109
:105530005FF0000318460AF8034008F8034009F832
:105540000340F454FC54FFF7B1FF5B1C022BF1DB6A
:105550002C706C702878401CC0B22870142839D97F
:105560002C701D4D0023AD1C05F1020BE95C59B3F5
:105570001BF8030020B3F25C8A4202D1FA5C82423B
:105580000AD00AF80340F154F8544900084409F8D5
:105590000310400008F803001AF803105046491C95
:1055A000CAB20AF8032018F803108A4200D9C4547A
:1055B0001AF8030019F80310884205D2C00703D077
:1055C0001846FFF78DFF02E01846FFF76FFF5B1CE0
:1055D000022BCBDBBDE8F08F6C00002038B54FF418
:1055E000A06001F02DF91E21012002F065F82520B0
:1055F0008DF8000001248DF801408DF802408DF8EF
:105600000340684601F0EAF82621012002F054F830
:1056100026208DF800008DF801408DF802408DF8AD
:105620000340684601F0DAF82E21012002F044F828
:1056300027208DF800008DF801408DF802408DF88C
:105640000340684601F0CAF83621012002F034F820
:105650000E208DF800008DF801408DF802408DF885
:105660000340684601F0BAF83D21012002F024F819
:105670000C208DF800008DF801408DF802408DF867
:105680000340684601F0AAF81E208DF800008DF84E
:1056900001408DF802408DF80340684601F09EF805
:1056A0001D208DF800008DF801408DF802408DF826
:1056B0000340684601F092F81C208DF800008DF838
:1056C00001408DF802408DF80340684601F086F8ED
:1056D00028208DF8000002208DF802008DF803408C
:1056E000684601F07BF838BD86B0DFF830C200DFD5
:1056F0008B4DA86001F03CFF002002F0D1FCFFF7C9
:105700000BF8884FB8B988A1012002F00BFA1326D4
:105710003C463220DFF820C200DF02212046FFF79E
:10572000A7FD00287ED0002202212046FFF7ABFD16
:10573000761EF6B2EDD201F0D5FE01F0B5FFFFF70F
:1057400039FE7EA1012002F0EDF9824C0120A11C5E
:1057500002F0E8F9628980A1684602F0C7FF694655
:10576000012002F0DFF9D4F812207DA1684602F092
:10577000BDFF6946012002F0D5F902213C463846BA
:10578000FFF776FD00285AD0002202212046FFF7BD
:105790007AFD0023754A76497648DFF8DCC100DFE0
:1057A0007649086002212046FFF762FDD8B3002247
:1057B00002212046FFF767FD0023714A71497248B4
:1057C000DFF8B4C100DF7149086002212046FFF70D
:1057D0004FFD48B3002202212046FFF754FD02216D
:1057E0002046FFF745FD70B300220221A146204666
:1057F000FFF749FD40F2C711072001F05DFF03F0FC
:105800000FFB634FDFF88C81DFF88CA100240120AF
:10581000DFF824C100DF3878012819D0022817D01A
:10582000464602E009E00CE00EE098F800202AB3BA
:105830009AF80000522849D050E0012274E7012272
:10584000A3E70122B4E701E00122C4E70122CCE78B
:1058500040F214525149524800F0A0FE061E0ADDE3
:10586000504844844D4884553878012807D0314643
:105870004A4802F09FFC387802281FD035E0FFF735
:105880007FFD02214846FFF7F3FC98B10022022178
:105890004846FFF7F8FC3146404802F08BFC0221F5
:1058A0004846FFF7E5FC38B1002202214846FFF7E1
:1058B000EAFCE0E70122EAE70122F6E798F80010A7
:1058C000464691B1344802F03FFE0DE09AF80110CF
:1058D000542903D19AF802002B2818D02E49002011
:1058E00003F0D6F98AF8004034700020FFF712FE6A
:1058F000FFF770FBDFF8B0C000DF2969884286D966
:105900006430286102F092F801F05CFD7FE72248E4
:1059100001F056F901202870E4E70000419B0008DF
:10592000380000200008014073466C61736820460F
:1059300061696C656421000041920008200D0A4DE8
:1059400061696E205461736B205374617274210D10
:105950000A000000220C00205F5625640D0A00009A
:1059600050534E3D256C750D0A0000006823002041
:105970000420030039640008F5980008580000204E
:10598000881C002003E0060061610008540000202C
:105990001800002019000020280600201401002013
:1059A000B026002088260020A99800080348026835
:1059B0000348018803A002F075FEFEE744000020C2
:1059C0003C0000200D0A5B4D4D485D463D25642C92
:1059D0004C3D256C7500000010B540F21454224671
:1059E0000349044800F0DAFD0028F8D110BD00009A
:1059F00014010020B02600200EB5FFF7EDFF4FF494
:105A00007A60009002AB01AA07A10AA000F0DCFABC
:105A1000012804D0022804D04FF0FF300EBD002032
:105A20000EBD01200EBD00004F4B7C4552524F521F
:105A30000000000041542B514944454143543D313D
:105A40000D0A000010B588B00446FFF7C5FF2346D5
:105A50000CA2142101A802F035FE40F24C40009047
:105A600007AB06AA0BA101A800F0AEFA012805D0E9
:105A7000022805D04FF0FF3008B010BD0020FBE732
:105A80000120F9E741542B5149434C4F53453D25E3
:105A9000640D0A004F4B7C4552524F5200000000EB
:105AA00010B588B00446142101A8FEF720FC40F28E
:105AB0004D11022001F000FEFFF78EFF4FF49670AB
:105AC000009007AB06AA0DA112A000F07DFA0128F4
:105AD00003D04FF0FF3008B010BD0021069A082017
:105AE000135C202B04D96354401C491C1C28F7DB91
:105AF0001C2801D00120EEE70020ECE72B514343A6
:105B000049443A207C2B434D45204552524F523A4E
:105B10002000000041542B51434349440D0A00002A
:105B20003EB504464FF47A60009002AB01AA10A182
:105B300011A000F049FA012816D102980A2813DDB5
:105B400001980021C2792C2A03D0027A2C2A02D093
:105B500002E0C17100E00172801DFEF71CFCC72845
:105B600002D8207000203EBD4FF0FF303EBD000047
:105B70002B4353513A00000041542B4353510D0A1B
:105B80000000000000B589B0142101A8FEF7AFFBAA
:105B900040F26B11022001F08FFDFFF71DFF4FF463
:105BA000FA70009007AB06AA09A110A000F00CFA49
:105BB000012805D0022805D04FF0FF3009B000BD04
:105BC0000020FBE76420DFF830C000DF0120F5E7AC
:105BD0002B4350494E3A2052454144597C2B434D6A
:105BE00045204552524F523A0000000041542B4389
:105BF00050494E3F0D0A00004192000870B58EB02A
:105C00000C4605460B281EDC03461CA2142102A8E4
:105C100002F058FD2B461EA2142107A802F052FDE7
:105C20004FF0FF364FF4967522E000BFFFF7D4FE29
:105C30000CAB01AA07A902A8009500F0C5F901283C
:105C400004D0022816DB01200EB070BD05222C21E5
:105C5000019803F0A5FF019008B1401C0190007865
:105C6000312809D03028EED06420DFF83CC000DFB6
:105C7000641EDBD23046E7E70020E5E741542B51B4
:105C80004953544154453D312C25640D0A00000010
:105C90002B514953544154453A25642C7C4F4B7C3D
:105CA0004552524F5200000041920008F8B50121C0
:105CB0001C2001F009FB10208DF8030003208DF853
:105CC0000200254F4025ADF8005069463846FFF7E1
:105CD00051FA8026ADF8006069463846FFF74AFA67
:105CE0000224ADF8004069463846FFF743FA1BA18D
:105CF000012001F017FF184F14373C603D603E60F3
:105D00003220DFF868C000DF3E1F34603220DFF849
:105D10005CC000DF35606420DFF850C000DF3D600C
:105D2000C820DFF848C000DF02F068FA142000F055
:105D3000F1FB0F4D30B16C700EA1012001F0F2FEAD
:105D40000120F8BD10A1012001F0ECFE00F0CEF919
:105D5000012068700020F8BD000C01404D6F6465A3
:105D60006D20496E69742E2E2E0D0A004192000896
:105D7000882600204D6F64656D2063616E27742056
:105D80006F70656E210D0A004D6F64656D2069733B
:105D9000206F70656E6564210D0A00000EB5FFF777
:105DA0001BFE0948009002AB01AA08A10AA000F05E
:105DB0000BF9012804D0022804D04FF0FF300EBDAB
:105DC00000200EBD01200EBDF04902004F4B7C4566
:105DD00052524F520000000041542B51494143544C
:105DE0003D310D0A00000000F0B5B1B01D46164669
:105DF0000F4604460B2829DCFFF7EEFD0097CDE99E
:105E00000165234613A2782103A802F05BFC03A9D5
:105E1000012001F087FE234617A2322121A802F0BB
:105E200051FC4FF4FA6000902FAB2EAA21A903A8D1
:105E300000F0CAF8012805D0022807D04FF0FF3043
:105E400031B0F0BD2E98C07A302801D00120F7E79C
:105E50000020F5E741542B51494F50454E3D312C20
:105E600025642C222573222C222573222C25642CB8
:105E7000302C310D0A0000002B51494F50454E3A4D
:105E80002025642C7C4552524F5200003EB5FFF74E
:105E9000A3FD40F21450009002AB01AA0BA10FA089
:105EA00000F092F8104C002240F22551204602F0FA
:105EB00054F80021204602F018F84FF49670DFF8ED
:105EC0002CC000DF0A49022008603EBD504F5745F4
:105ED00052454420444F574E0000000041542B517E
:105EE000504F57440D0A00000048004041920008FE
:105EF000140C01400EB5FFF76FFD0948009002AB8E
:105F000001AA08A10CA000F05FF8012804D0022823
:105F100004D04FF0FF300EBD00200EBD01200EBD9D
:105F2000F04902002B51494143543A20312C317C35
:105F30004552524F5200000041542B5149414354A5
:105F40003F0D0A002DE9F0410646FFF79FFF052EA1
:105F500006DA1648DFF858C030F8160000DF20E0F7
:105F6000124D00242D1F41F270770A2E2C600EDA9C
:105F700005F10E0000EB460604E03846DFF830C0BD
:105F800000DF641C36F80A0CA042F6DC08E04FF48F
:105F9000B4763846DFF818C000DF641CB442F8DB82
:105FA0002C60BDE8F041FFF781BE00000400002036
:105FB0004192000810B50446FEF7C2F981B22046AE
:105FC000BDE8104002F0C0BA2DE9F0411D4616466A
:105FD0000F46069CFFF7EEFF23462A463146384619
:105FE000BDE8F04100F048BA70B5FEF76BFD1D4802
:105FF0000079012834D11C4C6078002830D0DFF8BB
:106000006CC000DFA16888422AD3DFF860C000DFDF
:106010003230A0602078164DC0EBC00101EB0010BB
:106020000026295CA9B128448178012911D1417841
:1060300011B9C01C00F07AF92078C0EBC00101EB67
:10604000001028444178491CC9B24170062900D388
:1060500046702078401C10F0FF00207000D02670A1
:1060600070BD0000882600208C000020A998000840
:106070008530002002F068BA70B590B014460E4624
:1060800005460B2802D9012010B070BDFFF7A4FC13
:106090002B460FA2322101A8009402F013FB01A9A4
:1060A000012001F03FFD4FF47A7000900FAB0EAA73
:1060B0000CA101A8FFF788FF012802D04FF0FF30A4
:1060C000E2E721463046FFF7D5FF0020DCE700007D
:1060D00041542B514953454E443D25642C25640DB4
:1060E0000A0000003E7C4552524F52003EB500244B
:1060F0004FF49675FFF770FC02AB01AA06A107A04A
:106100000095FFF761FF012804D0641C032CF1DB2C
:1061100001203EBD00203EBD4F4B000041544530A4
:106120000D0A000030B50446012213E07C2B14D088
:1061300005789D4203D10BE07C2B05D0491C0B78E0
:10614000002BF9D1002030BD491C2046521C01E033
:10615000401C491C0B78002BE8D1104630BD0000D4
:1061600086B040F2C521082001F0A6FA49A101201D
:1061700001F0D8FC26214D48FEF7B9F8012000F0C7
:1061800069FB00F023FB494C022501276570A570CF
:10619000E57025716571A571FFF788FD20B144A1F7
:1061A000012001F0BFFCFEE7E7710026FFF7EAFCE3
:1061B00010B1761C142EF9DB142E17D00025658142
:1061C000A77040A1012001F0ADFC18216846FEF740
:1061D0008EF800266846FFF763FCA0B16420DFF864
:1061E000F4C000DF761C052EF4DB1BE03AA1012091
:1061F00001F098FC6089FFF7A5FE60893228C6D2BD
:10620000401C6081C3E7052E0CDA3F48694606460C
:10621000FEF79DF830B1142269463046FEF784F847
:1062200001F0DCFB394EDFF8E8903A4F4FF6FF7A89
:1062300040F2145BA846307820B15046DFF894C095
:1062400000DFF8E70120DFF88CC000DF17485A466E
:106250002F49283000F0A2F9051E0CDDA4F8228099
:1062600009F805802A49012001F05CFCA9B2284800
:10627000FEF700FB04E003DA27A1012001F052FC45
:1062800038780228D7D0FFF7AFFE002000F0E2FAFE
:10629000D1E700004D6F64656D5461736B205374DA
:1062A0006172742E2E2E0D0A000000008826002038
:1062B00057696C6C206265207265626F6F74210D86
:1062C0000A0000004765742049434349442E2E2E9E
:1062D0000D0A00004192000853494D206361726429
:1062E000206E6F74207265616479217265626F6FD0
:1062F0007420616E6420636865636B206167616907
:106300006E210D0A00000000560D00205C000020E8
:1063100014010020180000204D6F64656D4D7367F7
:10632000427566204F766572210D0A002DE9F04313
:10633000A5B0814609208DF8000030208DF80100BD
:1063400000268DF802602D208DF8030036486C463B
:106350000425D0F8123035A2142120A802F0B2F999
:10636000002020AA02EB400312F810105B7809010C
:1063700001F0F00103F00F03194361556D1C401C3F
:1063800080B2ADB20628EDD32A4A4FF010085088EB
:10639000010A61556D1CA9B26054491C8DB2401CA4
:1063A0005080601907464146FDF7A1FF1E49384657
:1063B0004246C631FDF782FF1035ADB2601907467F
:1063C0004146FDF794FF184938464246D631FDF75D
:1063D00075FF1035A8B20C212154401C80B2221840
:1063E000D9F800301360D9F804305360D9F8081098
:1063F00091600C3081B200206A4603E0135C5E407D
:10640000401C80B28842F9D36654491C8AB280216C
:10641000684600F059FB82B269460120FFF72CFE66
:1064200025B0BDE8F0830000220C00202530313279
:10643000640000008C00002000210A48DFF828C01A
:1064400000DF4FF6FF7421460648DFF820C000DF6A
:10645000DFF81CC000DF01F039FFDFF818C000DFF3
:10646000F1E70000640000204996000889960008C2
:10647000F19A0008519B00082DE9FF5F1D469346E5
:106480000F46002640F2145ADFF86480DFF864906B
:1064900026E052461649184800F080F8041E15D030
:1064A0001ADDA9F822601249012001F03BFBC7F870
:1064B0000080CBF800400E480099FFF733FE00281B
:1064C00012D1A1B20A48FEF7D5F909E00120DFF8A0
:1064D0002CC000DF6D1E03E009A1012001F022FBAA
:1064E000002DD6D100203E6004B0BDE8F09F000032
:1064F0001401002088260020B026002041920008C8
:106500004D6F64656D4D7367427566204F564552F9
:10651000210D0A00FEB50546FFF75EFA0024642649
:1065200009E002AB01AA07A107A00096FFF74CFD06
:10653000012805D0641CAC42F3DB4FF0FF30FEBDF8
:106540000020FEBD4F4B000041540D0A000000002A
:10655000B0F5FA6F01DA00F5FA60022909D00429D2
:106560001AD0062918D0092916D00B2914D01F20BB
:106570007047810705D1642190FBF1F201FB120104
:1065800041B94FF4C87190FBF1F201FB120008B160
:106590001C2070471D2070471E2070472DE9F047D2
:1065A00016468A460446DFF8D0C000DF761E1FFA82
:1065B00086F98121052001F07FF8A08860B160880C
:1065C00004EB8000C788008967F30F0560F31F455F
:1065D0000020064601461EE0DFF8A0C000DF0020D4
:1065E000BDE8F087228EC2B1A38ED4F838C01CF863
:1065F00003C05B1C9BB2A386B4F82E80434500D336
:10660000A186521E2286484503D20AF800C0401CCB
:1066100080B2761CB6B2B742E4D86288521C92B2FD
:1066200062800A2A00D36180A288521EA2800AF8E2
:1066300000109A21052001F03FF8A8B2B04209D01D
:106640000FA1012001F06EFAA8B24442DFF82CC07D
:1066500000DF0AE04F450AD90FA1012001F062FADC
:10666000A8B24442DFF814C000DF2046B8E7DFF8E4
:106670000CC000DFA8B2B3E7F19A0008519B0008F4
:106680004D73675175657565416363657074204529
:1066900072723D2D320D0A004D7367517565756537
:1066A000416363657074204572723D2D310D0A009F
:1066B00030B500230380838043801C4600EB8405B3
:1066C000641C2B81EB800A2CF8DB8163002102E043
:1066D000846B6354491C9142FADBC28543868386EE
:1066E000038630BD2DE9F04704468088089D984612
:1066F000174689460A2801D328A105E0208EE18D9E
:106700002844884205D32AA1BDE8F047012001F0C2
:1067100009BA5C21052000F0CFFF2188608E04EBD0
:10672000810108812088602104EB8000C58005205C
:1067300000F0C2FF002006461AE000BF19F808105A
:10674000638EA26B08F101081FFA88F8D154B8458E
:1067500001D34FF00008618E491C89B26186E28D39
:10676000914200D36686218E491C401C218680B24E
:10677000A842E3D36A21052000F09EFF2088401C38
:1067800080B220800A2800D32680A0886F21401C78
:10679000A080BDE8F047052000F08EBF4D73675123
:1067A000756575652066756C6C210D0A000000002A
:1067B0004D736751756575652044617461427566F6
:1067C0006665722066756C6C210D0A0028210148EF
:1067D000FDF78DBD5C2B00207047000070B50F23C6
:1067E000C47801780122F4B1144C2468457804F48B
:1067F000E064C4F5E064240AC4F10406E34084784C
:10680000B5401C402C4301F1E021230181F8003404
:10681000007800F01F018A404009800000F1E0206C
:10682000C0F8002170BD01F01F00824048098000BF
:1068300000F1E020C0F8802170BD00000CED00E008
:106840000249084302490860704700000000FA0549
:106850000CED00E02DE9F047002500285CD1DFF8C1
:10686000C0C100DF6F494A68821A642A54D96E4C4D
:1068700048606E4F207802264FF0040A4FF003095B
:106880004FF00108062847D2DFE800F0032C4860EB
:1068900090A467A1012001F045F9A671FFF772F9F4
:1068A00050B101280FD0A6702089401C80B22081F1
:1068B000052831D925810EE0258184F80280E58103
:1068C0004046658181E02581A670A089401C80B288
:1068D000A081142820D96089411C6181BDE8F0475E
:1068E000FFF730BB55A1012001F01CF94E48A671FD
:1068F0002030FFF715F970B9258194F82000801E2B
:106900001E2801D265813CE0E089401C80B2E08114
:10691000142801D9E5812570BDE8F08749A101203F
:1069200001F000F9A6715A2001F03CFE48B1E67072
:106930006089411C6181FFF705FB60890628EAD860
:10694000EAE784F8038084F800900FE040A101207A
:1069500001F0E8F8A671FFF721FA10B1012807D07D
:1069600022E084F8048084F800A025826581D3E7C2
:106970002671FFF741F818B1012804D0267108E00C
:1069800025822670C8E7208A401C80B22082032816
:10699000C2D925826089411C6181FFF7D3FA6089E1
:1069A0000628B9D96581B6E72671F3E72AA1012047
:1069B00001F0B8F8FFF79EFA18B1012807D03D7032
:1069C000F2E738780028A7D105202070A4E784F8E2
:1069D000009009E024A1012001F0A4F80A2101207F
:1069E000FFF70CF9012801D03D7095E7FEF740F95B
:1069F00048B101283D7010D020A1012001F092F88B
:106A000084F8009088E787F8008084F800A0BDE84B
:106A1000F04721A1012001F085B825A1EDE7000094
:106A2000A99800085C000020882600208D00002026
:106A30003C434152443E0D0A000000003C43535188
:106A40003E0D0A003C435245473E0D0A000000003F
:106A50003C5044503E0D0A003C51554552595F5040
:106A600044503E0D0A0000003C51554552595F55B7
:106A7000534F434B45543E0D0A000000436F6E6E6A
:106A8000656374207365727665722074696D656FD5
:106A90007574210D0A000000436F6E6E65637420EB
:106AA000736572766572204F6B210D0A000000003D
:106AB000436F6E6E656374207365727665722066CF
:106AC00061696C210D0A0000F0B5034600242046E0
:106AD00006E01D5C7E2D01D07D2D00D1641C401C84
:106AE0009042F6DB1019801C884201DD0020F0BDC9
:106AF00019187E2501F8015C811E02267D240127DC
:106B00000BE000BF13F802C0BCF17E0F10D0BCF147
:106B10007D0F0FD003F801C0491E521E002AF1DC80
:106B20001A787E2A0DD07D2A0DD05A541D70F0BDE2
:106B30005E5400E05F54A1F1010C891E03F80C4083
:106B4000EBE75E5400E05F54491E5C54EEE770B51D
:106B500002787E2A04D1421812F8012C7E2A02D033
:106B60004FF0FF3070BD0024421C25460346491EED
:106B70001AE006787E2E07D07D2E0AD0401C521CCB
:106B800003F8016B641C0EE084B90124401C521C04
:106B90000AE01678012E04D0022E09D06FF0020010
:106BA00070BD7D2605E06D1C8C42E2DB284670BD81
:106BB0007E26801C921C03F8016BA41CF3E70000E6
:106BC0002DE9F04FBBB005464422F9492AA8FDF74C
:106BD00075FB00273C467C21072000F06DFD2AAEA6
:106BE00056F82400641C00780028F9D18021072081
:106BF000641E00F061FD002309E000BF56F8232069
:106C0000E81C2DE090F800C0614527D05B1CA34232
:106C1000F4DB9521072000F04FFDA3427ED0E54C28
:106C20004FF0000804F16E0002901830019005F159
:106C30000A0004F19E0604F1C60B04F1D60A04F121
:106C4000E6090090102B62D2DFE803F00E141C312D
:106C5000777F83B6FDFCFBFAF9F8F7F6401C521C6F
:106C600011780029CED1D4E7D3A1002000F05AFF3B
:106C7000022004E0D3A1002000F054FF0120FDF722
:106C8000A9FF44E0D24C94F8200040B1D1A10020EB
:106C900000F048FF84F8208000F0A0FE37E0D2A189
:106CA000002000F03FFF012084F82000F4E704AA50
:106CB000D2A12846FEF7ECFA401E132801D3D0A13A
:106CC00022E004A90298FDF75DFB04AAD3A128469F
:106CD000FEF7DEFA401E132801D3D2A114E004A966
:106CE0000198FDF74FFB04AAD6A12846FEF7D0FA7B
:106CF000401E132801D3D5A106E004A93046FDF7B4
:106D000041FB00F073FED9A1002000F00BFF40F220
:106D10006711072000F0D0FC287800E00AE0542832
:106D200008D168784D2805D1D5A001F0BBFC022020
:106D3000FDF750FF3BB0BDE8F08F0096DDE9013272
:106D4000D3A104A801F0D2FC96E26389A289D6A15E
:106D5000FEE0984A34F8423F1A32D8A104A801F064
:106D6000C5FC04A9002000F0DDFED84E2288B078D2
:106D7000F1788DE8070073783278D5A104A801F086
:106D8000B5FC04A9002000F0CDFE8A4A638D443290
:106D9000D6A104A801F0AAFC04A9002000F0C2FEBC
:106DA000B079628DF1798DE8070073793279D3A1DA
:106DB00004A801F09BFC5FE204AAD6A12846FEF7D6
:106DC00067FA401E0A280ED204A8FDF7F1FA060061
:106DD00009D004AAD0A12846FEF75AFA401E0A2874
:106DE00003D3CFA190E7D6A18EE704A8FDF7E0FA80
:106DF0000746304602F0CCF8B84204D0D8A10020B3
:106E000000F090FE96E76B49C4F81260C4F8167063
:106E100041F8B68F3046A1F8048066490522B731A3
:106E2000A234FEF70DF8F820A0762320E076872024
:106E3000207754F8900C07E08EE085E064E060E095
:106E40003FE038E035E030E0010C6177010AA177DE
:106E5000E07700F0CBFD00F08BFB54F88C3C54F84D
:106E6000902CC1A104A801F041FC04A9002000F06D
:106E700059FEE07D627E217E8DE80700A37D627D64
:106E8000BEA104A801F032FC04A9002000F04AFED3
:106E9000207FE37FA27F617F8DE80F00E37EA27EEB
:106EA000BEA104A801F022FCE6E1D4F81220C4A19E
:106EB00003E000F085FE5A46C4A104A801F016FCC8
:106EC000DAE110215846FDF712FA0024464604E0A4
:106ED000285D0D2800D12E55641C2846FDF730FA98
:106EE000A042F5D80098FDF72BFA0246102800D3EF
:106EF0000F2258460099FDF7E1F900F077FDB6A1A1
:106F000002E75246B8A1D8E710215046FDF7EFF945
:106F10000024464604E0285D0D2800D12E55641C4F
:106F20002846FDF70DFAA042F5D80098FDF708FABB
:106F30000246102800D30F2250460099FDF7BEF9F3
:106F400000F054FDABA1DFE6B4F80E314A46ADA126
:106F500004A801F0CBFB8FE104AAAFA12846FEF7FD
:106F600097F9401E132801D3ACA1CDE604A94846E9
:106F7000FDF7EDF920B104A94846FDF703FA012712
:106F800004AAADA12846FEF783F9401E052801D3C7
:106F9000ABA1B9E604A8FDF7FEF9B4F80E118842DA
:106FA00005D004A8FDF7F7F9A4F80E0159E157E15F
:106FB000E89C0008220C002052542B544D3A4F4BB1
:106FC0000D0A000052542B54473A4F4B0D0A000053
:106FD000320D002052542B44454255474C4F473AFE
:106FE0004F46460D0A00000052542B444542554777
:106FF0004C4F473A4F4E0D0A0000000041504E00E2
:1070000052542B5353494D3A4641494C5B41504EE3
:1070100020496E76616C69645D0D0A004E414D45F4
:107020000000000052542B5353494D3A4641494CFD
:107030005B4E414D4520496E76616C69645D0D0A79
:1070400000000000504153530000000052542B53E5
:1070500053494D3A4641494C5B5041535320496E88
:1070600076616C69645D0D0A000000005365742050
:1070700053494D20496E666F204F4B210D0A000089
:107080002D2D2D2D544D2D2D2D2D0D0A00000000E0
:1070900041504E3D25733B5553523D25733B504166
:1070A00053533D25730D0A00485665723D256420F3
:1070B000535665723D25640D0A00000041707053FF
:1070C0003A25733A25640D0A0000000030000020C4
:1070D00053657276657249503A25642E25642E25D3
:1070E000642E25643A25640D0A000000466F746121
:1070F000533A25733A25640D0A000000466F746107
:1071000049503A25642E25642E25642E25643A259F
:10711000640D0A0050534E00414B455900000000D9
:1071200052542B53455449443A4641494C5B414BD8
:10713000455920496E76616C69645D0D0A00000056
:1071400052542B53455449443A4641494C5B5053A1
:107150004E20496E76616C69645D0D0A0000000086
:1071600050534E3D300D0A0050534E3D256C750D69
:107170000A414B45593D256C750D0A0044657669F9
:10718000636549443D2578253032782530327825AD
:10719000303278253032780D0A0000004D41433DF1
:1071A000253032582E253032582E253032582E2593
:1071B0003032582E253032582E253032580D0A00E4
:1071C00050534E3D256C640D0A00000052504E4154
:1071D0004D453D25730D0A0052542B53504E414DE1
:1071E000453A4F4B0D0A000052444E414D453D2556
:1071F000730D0A0052542B53444E414D453A4F4BA8
:107200000D0A000052542B52415345523D25732C18
:1072100025640D0A000000004950000052542B5311
:10722000415345523A4641494C5B495020496E769C
:10723000616C69645D0D0A00506F7274000000009B
:1072400052542B53415345523A4641494C5B506F7F
:10725000727420496E76616C69645D0D0A000000ED
:107260000FB100F0C3FBB4F80E0100904B4603A22F
:10727000962104A801F026FA04A945E552542B539F
:10728000415345523A49503D25733B506F72743D0E
:1072900025640D0A00000000044A0029516901D04C
:1072A000014300E08143516170470000001002403B
:1072B000044A0029D16901D0014300E08143D16132
:1072C0007047000000100240044A0029916901D073
:1072D000014300E0814391617047000000100240CB
:1072E0000248416A41F080714162704700100240DB
:1072F00030B5224A5168224B11F00C0103D0042909
:1073000003D0082903D0036016E01E4913E051683A
:10731000536801F470114FF0020413F4803F04EB42
:10732000914104D053689B0303D5174B02E0174BE0
:1073300000E0144B5943016051680F2303EA111117
:10734000134B5C5C0168E14041605468072505EA25
:1073500014241C5D21FA04F48460546805EAD424E2
:107360001B5DD940C1605268032303EA9232084B87
:107370001B1F9A5CB1FBF2F1016130BD00100240AD
:1073800000127A00001BB700808D5B0000093D00F1
:107390009C0000200246002053090949012B0BD014
:1073A000022B0BD0D1F8241002F01F0201239340CE
:1073B0000B4200D0012070470968F5E7096AF3E73E
:1073C0000010024010B5DFF868C000DF194B187AD2
:1073D000401CC0B218723B2825D900201872D979F8
:1073E000491CC9B2D9713B291DD9D8719979491C59
:1073F000C9B29971172916D9987119791868FFF7C8
:10740000A7F85979491CC9B2597188420BDA012091
:1074100058711979491CC9B219710C2903D918710D
:107420001868401C1860DFF810C000DF10BD0000B5
:10743000F19A000880000020519B000810B5044616
:10744000DFF894C000DF2078DFF894C0000900EB7B
:107450008000410021480160227802F00F021144AF
:1074600001F5FA6101606178090901EB81014900C8
:107470000171627802F00F0211440171A1780909CB
:1074800001EB810149004171A27802F00F02114421
:107490004171E178090901EB810149008171E278CC
:1074A00002F00F02114481712179090901EB810178
:1074B0004900C171227902F00F021144C171617952
:1074C000090901EB810149000172627902F00F02A2
:1074D0001144017200DF10BDF19A00088000002005
:1074E000519B000870B560220021124800F02AF973
:1074F000104C114D2068A84202D1E06DA84217D06F
:107500000EA1012000F00EFB60210A48FCF7EFFEFF
:1075100044F8045B4FF40050A5656061012060777A
:107520000520A0773C20E077BDE8704000F056BA17
:1075300070BD0000320D002005563412526573658F
:107540007420446576696365436F6E666967210DD3
:107550000A00000030B500231C4606E0055BCD5450
:107560005B1C2D0ACD545B1CA41C9442F6DB30BD81
:107570002DE9F047DFF8E4A04FF488794A46364910
:107580005046FFF7E7FF344C47F60157344E20884A
:1075900040F2B6454FF00208B84203D1D4F8C20019
:1075A000B0424DD049462C48FCF7A1FE27802DA3C0
:1075B0002EA20821A01C01F085F86581A4F80C809A
:1075C0000120A073E0732074234829A327A2282157
:1075D0001A3001F077F844F64B20A4F842001E4818
:1075E00027A322A22821443001F06CF842F2B130E6
:1075F000A4F86C00184826A31CA218216E3001F0D4
:1076000061F8154824A319A21821863001F05AF810
:10761000114821A315A218219E3001F053F8C4F897
:10762000C2604A460C49504600F0FAFF0A481CA1C5
:10763000C630FCF7A7FE08481AA1D630FCF7A2FE18
:1076400008A30AA20821A01C01F03CF86581A4F857
:107650000C80BDE8F0870000220C002000F000083C
:10766000545C1A0552543233314100002573000036
:1076700034372E3130362E3234322E313400000081
:10768000666F74612E7274756F6C2E636F6D00007F
:10769000636D6E6574000000636172640000000039
:1076A0005A524B004D32300008225102014800F07E
:1076B00049B8000030000020014A9080D160704736
:1076C000380000200029018802D041F0400101E08B
:1076D00021F040010180704710B5074C1021204671
:1076E000FDF7CDFD062000F05FF92046BDE8104013
:1076F0001021FDF7C6BD00000008014070B504036D
:10770000FFF7EAFF00F084F80D4D10212846FDF741
:10771000B6FD202000F048F9C4F3074000F044F91A
:10772000C4F3072000F040F9E0B200F03DF9102169
:107730002846FDF7A6FDBDE8704000F069B80000DE
:10774000000801402DE9F041144F0C46054616464D
:1077500010213846FDF793FD0B2000F025F9C4F306
:10776000074000F021F9C4F3072000F01DF9E0B252
:1077700000F01AF9FF2000F017F92870002405E046
:10778000FF2000F011F92855641CA4B2B442F7D3CD
:107790003846BDE8F0411021FDF773BD00080140F7
:1077A0002DE9F0410E4E10213046FDF768FD9F2077
:1077B00000F0FAF8FF2000F0F7F80546FF2000F08F
:1077C000F3F80446FF2000F0EFF80746102130469A
:1077D000FDF757FD280440EA04203843BDE8F08156
:1077E0000008014070B5094D10212846FDF747FDFE
:1077F000052000F0D9F8FF2000F0D6F8044610214B
:107800002846FDF73EFD204670BD000000080140FF
:107810002DE91040FFF7E6FFC007FBD110BD0000C7
:107820002DE9F05FC1F30B060F0BC6F580548846B7
:1078300082461546A24200D81446DFF87C903903F0
:107840008B464FF480521C48FFF77CFF002006E077
:10785000321819F80210FF2903D1401C80B2A0424F
:10786000F6D3A04222D23846FFF748FF00204A460E
:1078700006E000BF1AF800108319401CD15480B2F2
:10788000A042F7D359464FF480520B4800F016F847
:10789000A5420FD0281BA244A044002685B24FF475
:1078A00080547F1CA542CAD82C46C8E722464146D0
:1078B0005046EBE7BDE8F09F9C3000202DE9F041F9
:1078C0000746C8B2C0F580740E461546A24200D8DD
:1078D00014464FF4807822463146384600F00EF8C0
:1078E000A54208D0281B2744264485B24446A54219
:1078F000F1D82C46EFE7BDE8F08100002DE9F0411A
:1079000015460C460646FFF7E7FE124F1021384693
:10791000FDF7B5FC022000F047F8C4F3074000F083
:1079200043F8C4F3072000F03FF8E0B200F03CF861
:10793000002404E0305D00F037F8641CA4B2AC42CF
:10794000F8D310213846FDF79CFCBDE8F041FFF765
:107950005FBF0000000801400246002012890A4271
:1079600000D001207047808970478181704730B511
:1079700002884C8802F441530A88CD8822438C88BF
:107980002C4322430C8922434C8922438C89224375
:10799000CC8922431A430280828B22F400628283C4
:1079A000098A018230BD000070B50B4C05460221EA
:1079B0002046FFF7D1FF0028F9D029462046FFF7DF
:1079C000D4FF01212046FFF7C7FF0028F9D0204649
:1079D000FFF7C9FFC0B270BD003001406022002136
:1079E0000148FFF71DBF0000320D002010B5012037
:1079F00080F310884FF488720349044800F010FEA9
:107A0000002080F3108810BD220C002000F0000838
:107A10008B185B00FF2B05DC022803D2024B1954A4
:107A2000991C0A54704700006E00002001F0AEB9A6
:107A300009291DD2DFE801F005080A1315180D0FFA
:107A400011000022114611E0002200E00122012174
:107A50000CE00622FBE7062204E0062205E01422E1
:107A6000F5E71422022101E014220321FFF7D0BF21
:107A7000704700000CB50021274801910091026871
:107A800042F4803202604FF4A063026802F40032D4
:107A90000092019A521C0192009A12B9019A9A42DC
:107AA000F3D10268920333D5012100911B490A6882
:107AB00042F010020A600A6822F003020A600A68B3
:107AC00042F002020A6041684160416841604168D9
:107AD00041F480614160416821F47C11416041685A
:107AE00041F488114160016841F0807101600168D2
:107AF0008901FCD5416821F003014160416841F0F2
:107B0000020141604168C1F381010229FAD10CBD33
:107B1000034800910170FEE700100240002002407F
:107B2000AC00002070B50D460D4991F8201009B940
:107B3000012813D00B48007800280FD10A484FF4D1
:107B4000807404602846FCF7FBFB0146A04200DD80
:107B500021462846BDE8704000F02CBB70BD0000F7
:107B6000320D002018000020100801400F4810B509
:107B7000016841F00101016041680D4A1140416016
:107B800001680C4A11400160016821F48021016004
:107B9000416821F4FE0141604FF41F018160FFF74D
:107BA00069FF06490448086010BD0000001002404B
:107BB0000000FFF8FFFFF6FE0040000808ED00E0BF
:107BC00003490120487003A1FFF7ACFFFEE7000066
:107BD0003800002053797374656D207265626F6F91
:107BE00074206E6F77210D0A0000000010B501218E
:107BF0008C07204600F00EF8002805D02046BDE88E
:107C00001040012100F003B810BD70477047C94310
:107C10000182704702460020138A92890B4202EAD1
:107C2000010202D0002A00D001207047F8B5374D7C
:107C300040F22441284600F071F9354C20B12888E3
:107C4000E081281D0088E08140F225563146284613
:107C500000F064F970B3284600F0EEF98DF80000EA
:107C60003146284600F03BF92078022804D060789D
:107C7000002138B12182F8BD9DF80010254800F0A0
:107C8000DFF917E09DF80030234A208A1354401C86
:107C900080B220821378522B1BD0892B2DD02182C9
:107CA0001170608A632802D36182A17061709DF8AF
:107CB0000000E0700821284600F029F90128DAD1F7
:107CC000284600F0B9F92846BDE8F840082100F040
:107CD00003B9022802D35378542B04D1032804D3C8
:107CE00092782B2A01D02182DBE7E2780D2AD8D1C5
:107CF0009DF800200A2A07D0D3E70328D1D3927831
:107D0000D21CE2819042CCD36070ECE70038014095
:107D1000180000200048004028060020F8B5304C2C
:107D200040F225552946204600F0F8F8F0B32046E9
:107D300000F082F98DF800002A4A1078012803D05B
:107D4000D08A002158B130E02946204600F0C7F81B
:107D50009DF80010BDE8F840234800F071B99DF887
:107D600000602248938AE52BC65401D25B1C9382A3
:107D700013790D2B1CD19DF800300A2B18D10378F4
:107D8000242B12D1C378522B0FD103794D2B0CD158
:107D90004379432B09D1164B968AD6821F7847F038
:107DA00001071F7059709970815500E007E09182BA
:107DB0009DF8000010712946204600F090F8082137
:107DC000204600F0A4F8012808D1204600F034F93C
:107DD0002046BDE8F840082100F07EB8F8BD00005C
:107DE0000044004018000020003801403C0B0020F7
:107DF000382B0020F8B5204C40F225552946204666
:107E000000F08CF810B3204600F016F98DF8000051
:107E10001A4A1078022828D013894FF496618B42B1
:107E20000DD29DF80060164FD0883E54401C80B2A1
:107E3000D080884201D30020D0805B1C1381114880
:107E400001F0D6F82946204600F049F808212046DE
:107E500000F05DF801280ED1204600F0EDF8204634
:107E6000BDE8F840082100F037B89DF8001006483A
:107E700000F0E6F8E6E7F8BD0048004018000020F2
:107E80008C060020640000200038014002494FF4B5
:107E900080700860FFF7CABE1408014010B54FF4A7
:107EA00000542046FCF79EFF01280CD10003FCF78C
:107EB0000FFF2046FCF700FF00210348FCF714FFEA
:107EC00002490020487110BD440002401800002003
:107ED000FFF724BFFFF78EBFC943018070470A0A2E
:107EE00001219140C943018070470029818902D056
:107EF00041F4005101E021F4005181817047002AD2
:107F0000828A01D00A4300E08A4382827047024697
:107F1000002012880A4200D00120704730B501F0DD
:107F20001F0201240025C1F3421304FA02F2012BBF
:107F30000FD0022B0FD0838A4FEA11210088134201
:107F400004FA01F400EA040001D000B1012528463A
:107F500030BD8389F0E7038AEEE710B5C1F3421321
:107F600001F01F040121A140012B07D0022B07D0F3
:107F70001430002A026805D00A4304E00C30F8E708
:107F80001030F6E78A43026010BD000030B50446A9
:107F9000008A85B00D464CF6FF710840E988014320
:107FA0002182A1894EF6F3100140A8882A89104346
:107FB0006A890A431043A081A08A4FF6FF41084016
:107FC000A9890143A1826846FFF792F919488442C2
:107FD00001D1039800E00298A189090400EBC001D7
:107FE00001EB0010296801D5490000E08900B0FBD1
:107FF000F1F06422B0FBF2F109010B096FF01805F2
:108000006B4300EB8300A3891D044FF0320306D5B8
:1080100003EBC000B0FBF2F000F0070005E003EB5B
:108020000010B0FBF2F000F00F000843208105B013
:1080300030BD0000003801408088C0F30800704760
:10804000C1F308018180704710B501218CB008464A
:10805000FFF722F90F4C2046FCF752FE0E48009025
:108060000E480021CDE901016420CDE90301802003
:10807000CDE905018001CDE9081007910A91694613
:108080002046FCF7BFFE01212046FCF72DFE0CB078
:1080900010BD0000580002400438014028060020AE
:1080A000F0B5064685B0012144F20400FFF70CF953
:1080B0004FF40070ADF8000018208DF80300394D22
:1080C00003248DF8024069462846FDF753F8AF15A2
:1080D000ADF8007010208DF803008DF8024069465D
:1080E0002846FDF747F82815ADF8000048208DF820
:1080F00003008DF8024069462846FDF73BF800244E
:108100004FF4E1300190ADF80C400C20264DADF855
:108110000840ADF80E00ADF80A40ADF8104001A9D6
:108120002846FFF733FF01212846FFF7DEFE4021F6
:108130002846FFF7D1FE002240F227712846FFF7BC
:108140000CFF300040F2255140F224464FF001026E
:1081500028461DD0FFF701FF002231462846FFF7D1
:10816000FCFE002240212846FFF7C9FE00228021A4
:108170002846FFF7C4FE00210C48FCF7B5FD0C486B
:1081800044824470447107481430076005B0F0BD64
:10819000FFF7E3FE002231462846FFF7DEFEFFF739
:1081A00053FFECE70008014000380140580002404E
:1081B000180000202DE9F04180460E484FF48077EA
:1081C0000E46076000240C4D0CE000BF18F80410A8
:1081D0002846FFF735FF40212846FFF798FE002884
:1081E000F9D0641CB442F1DB0248001D0760BDE811
:1081F000F0810000100801400038014030B52E48E1
:1082000085B00024C4800481448140F24C422B4953
:108210002B48FEF74DFA01210820FFF755F8012100
:108220008804FFF745F84FF40060ADF810004820CF
:108230008DF813000320234D8DF8120004A9284661
:10824000FCF798FF2815ADF8100018208DF81300E2
:1082500004A92846FCF78EFF4FF4E130ADF8044046
:108260000090ADF80640ADF80840ADF80C400C2089
:10827000154CADF80A0069462046FFF787FE4021FD
:108280002046FFF729FE002240F227712046FFF723
:1082900064FE012240F225512046FFF75EFE0022D7
:1082A00040F224412046FFF758FE01212046FFF707
:1082B0001CFE05B030BD000018000020EC26002098
:1082C000B0260020000C0140004800402DE9FF5F6F
:1082D000D5210420FFF7F0F9924CDFF84CB2DFF81B
:1082E0004C92208940F2AF4A40F225554FF49668EF
:1082F000012814D1002229465846FFF72EFEE788B0
:108300002689012229465846FFF727FE17B17F1E0E
:10831000B8B200E0504619F800003E2820D020896D
:1083200002281BD340F2AE4188424FF0000229469A
:108330005E46584630D9FFF710FE0022E280628187
:108340002281012229463046FFF707FE78A101204D
:10835000FFF7E8FBF4210420FFF7AEF9BDE8FF9F2B
:10836000009663894746424670497548FEF7BAF958
:10837000608900223044B0FBF7F107FB11006081F7
:1083800029465F465846FFF7E8FD20892946801BAD
:1083900020810122384696E0FFF7DFFDA346E788FB
:1083A0002489012229463046FFF7D7FD37B17F1EC9
:1083B0003804000C19F8001003D105E099F8AF1447
:1083C0005046401E80B200E050464A4619F8000070
:1083D0000D28C3D10A29C1D1022C07D0BBF80C004B
:1083E0005F46B0B10A2872D214307AE0BBF80A00B6
:1083F0005C46801CB0FBF8F208FB1200ABF80A00E8
:10840000002229463046FFF7A8FD2089801E2081E2
:1084100056E0132C3ED97889DFF828A18146002147
:10842000C446135C401C80B2604500D900201AF895
:108430000180984503D1491C89B20F29F1D30F2936
:1084400004D04B46E0466246009426E0401C80B2D1
:10845000604500D90020401C81B2614500D900214F
:10846000002001AB4FEA0C0812F801C0491C89B288
:1084700003F800C0414500D90021401C80B2042807
:10848000F2D3002119541846FBF785FF0004000CB5
:10849000B8819ED100947B89424624492848FEF742
:1084A00021F978890119B1FBF8F208FB12107881E3
:1084B000002229463046FFF750FD3889001B3881DD
:1084C000012229463046FFF748FD47E7FFE76428C9
:1084D00001D2153005E0B0F57A7F01D2163000E008
:1084E000173080B28442F0D300947B8942460F4912
:1084F0001348FEF7F7F878890119B1FBF8F208FB89
:1085000012107881002229463046FFF726FD38896F
:108510000122001B388129463046FFF71EFD00204E
:10852000B8811BE718000020004800408C0600209E
:108530005B527833427566204F7665725D0D0A0096
:10854000B0260020D69C00082DE9F0410E460746D3
:108550000024084D0AE0395D2846FFF771FD4021EF
:108560002846FFF7D4FC0028F9D0641CB442F2DBA3
:10857000BDE8F081004800400348026803480188D4
:1085800003A000F08FF8FEE7440000203C0000202C
:108590000D0A5B5546485D463D25642C4C3D256CD7
:1085A00075000000FEB500240646642515E0E007CE
:1085B00002AB01AA009507D00AA110A0FDF704FDA7
:1085C000002805DD0020FEBD0FA111A0FDF7FCFC79
:1085D0006420DFF848C000DF641CB442E7DB4FF0E2
:1085E000FF30FEBD2B435245473A20302C317C2BC7
:1085F000435245473A20302C3500000041542B436C
:108600005245473F0D0A00002B4353513A000000EA
:1086100041542B4353510D0A0000000041920008C1
:108620002DE9F0410E46054617462D210620FFF79D
:1086300043F872B6A5F10060B0F5803F30D2A805CE
:108640002ED132210620FFF737F8FCF7A5FC3421A4
:108650000620FFF731F82846FCF74AFC042801D031
:10866000372119E03B210620FFF726F800240AE015
:108670003119305D497800EB012081B22819FCF7EF
:1086800071FCA41CA4B2BC42F2D343210620FFF724
:1086900013F8FCF75FFC45210620FFF70DF862B6E2
:1086A000BDE8F0810FB4054B10B503A9044A029848
:1086B00000F066F810BC5DF814FB00005D8F000848
:1086C0000C0100200FB41CB50A46521ECDE9000271
:1086D00007A9054B6A46069800F052F8009A002157
:1086E00011701CBC5DF814FBE38B00080FB4084B41
:1086F00010B504A902AA039800F042F8044602A9A2
:10870000002000F079FA204610BC5DF814FB000050
:10871000F98B0008004870471001002002E008C8EB
:10872000121F08C1002AFAD170477047002001E0EB
:1087300001C1121F002AFBD1704710B5002A06DACA
:1087400022F00042D21D22F00703102203E0D21CC7
:1087500022F003030C2213B19C188C4201D9012092
:1087600010BD024401448360C0E90021C91AD01839
:10877000884202D810600246F9E70020106010BD60
:108780002DE9FF4F8DB00F460546002606E025284F
:108790000BD0DDE90F1290476D1C761C287800285D
:1087A000F5D111B03046BDE8F08F0024A246A146B5
:1087B0000122EC4900E0044315F8013F203B02FA96
:1087C00003F00842F7D128782A2810D06FF02F0242
:1087D0002878A0F13001092914D80AEB8A0102EBAC
:1087E000410144F0020400EB010A6D1CF0E701CFE7
:1087F0005FEA000A03D544F40054CAF1000A44F0C9
:1088000002046D1C28782E2817D115F8010F44F0AA
:1088100004042A280ED06FF02F022878A0F130012E
:1088200009290AD809EB890102EB410100EB010992
:108830006D1CF2E757F8049B6D1C28786C280FD04C
:1088400006DC4C2817D068280DD06A2814D104E023
:10885000742810D07A280FD10DE044F400140AE0F7
:1088600044F4801401E044F440146978814202D158
:1088700004F580146D1C6D1C2A786E2A1FD00CDC48
:10888000632A31D004DC002A8BD0582A11D1A3E00E
:10889000642A68D0692A0CD165E0732A2ED004DCE2
:1088A0006F2A73D0702A04D19BE0752A6FD0782A82
:1088B0006ED01046DDE90F129047761C50E1C4F3EC
:1088C0000250022806D0032809D0042801CF09D07D
:1088D000066045E101CFF117C0E9006140E101CF39
:1088E00006803DE106703BE117F8040B8DF80000AF
:1088F00000208DF80100EB46012003E057F804BB8F
:108900004FF0FF3061074FF0000102D40DE008F195
:108910000101884649450FDA8045F8DB1BF808104D
:108920000029F4D108E008F1010188468142FADB10
:108930001BF808100029F6D1DDE90F23AAEB080087
:108940008146214600F036F9304400EB080604E089
:10895000DDE90F121BF8010B9047B8F10108F7D2BF
:1089600021464846F7E00A21C4F302534FF0000BBA
:108970000891022B04D001CFC117032B09D00AE0C4
:10898000FF1D27F00707F7E8020108E032E01FE0CB
:1089900020E000B2C117042B01D140B2C117031E61
:1089A00071F1000307DA4FF0000CD0EB0C006CEB18
:1089B00001012D2302E0230504D52B238DF824305B
:1089C000012303E0E30701D02023F7E7984658E0AE
:1089D0000A2110E010210EE010204FF0000B08904B
:1089E0000CE010214FF0000B44F004044FF0080994
:1089F000089103E008214FF0000B0891C4F30253E3
:108A0000022B04D001CF0021032B06D006E0FF1D6E
:108A100027F00707F7E8020103E080B2042B00D13A
:108A2000C0B24FF0000823072BD5702A07D0DDF81D
:108A300020C08CF0100C5CEA0B0C05D00EE040233B
:108A40008DF82430012308E050EA010306D03023DA
:108A50008DF824308DF8252002239846DDF820C0BB
:108A60008CF0080C5CEA0B0C0BD150EA010301D12D
:108A7000630706D530238DF824304FF00108A9F1A3
:108A80000109582A04D038A20B9208AA0A920BE0D6
:108A90003AA2F9E75B46089AFBF797FC0B9B9B5CB5
:108AA0000A9A521E0A92137050EA0102F2D10A98F1
:108AB000ADEB000000F1200B600702D524F48034F8
:108AC00001E04FF00109D94502DDA9EB0B0000E000
:108AD000002000EB0B0141440890AAEB010AE003DF
:108AE00006D4DDE90F232146504600F063F8064422
:108AF0004FF0000908E009A911F80900DDE90F129B
:108B0000904709F10109761CC145F4DBE0030CD55F
:108B1000DDE90F232146504600F04CF8064404E0FE
:108B2000DDE90F1230209047761C0899481E089006
:108B30000029F5DC08E00A980A990078491C0A9196
:108B4000DDE90F129047761CBBF10001ABF1010B80
:108B5000F1DC21465046DDE90F2300F019F8064408
:108B60006D1C1BE6092801003031323334353637AD
:108B70003839616263646566000000003031323369
:108B80003435363738394142434445460000000009
:108B90002DE9F041044600251E461746880404D4FA
:108BA00005E039462020B0476D1C641EF9D52846E3
:108BB000BDE8F0812DE9F041044600251E469046AF
:108BC000C80301D5302700E02027880404D505E03C
:108BD00041463846B0476D1C641EF9D52846BDE8AD
:108BE000F0814A68002A06D00A68531C0B60107096
:108BF0004868401E486070470A68531C0B6010703C
:108C000070470000FEB5044600680090606801905F
:108C1000A068029094F8200094F82160002812D1F6
:108C20001A4F0025C5EBC50000EB0510395C31B1CA
:108C3000C1190C226846C91CFBF797FB20B16D1CBB
:108C400015F0FF05EED0FEBD94F82600704000023E
:108C500000F47F4194F825007040084301026FF052
:108C6000FF00014094F8240070400843010294F88A
:108C7000230070400843C5EBC50101EB05113944E1
:108C8000C1F80F0002208870FEBD00008530002072
:108C90002DE9FF410F780025CB1C892F03D001203F
:108CA00004B0BDE8F0818C78E41C944201D002202D
:108CB000F6E70024561E05E011F804C0641C8CEA97
:108CC0000505A4B2B442F7DB8C1814F8014CAC4291
:108CD00001D00320E4E78DF80C208DF80D704A7860
:108CE0008DF80E20002203AD03260BE0B2FBF6F454
:108CF00006FB14249F5C2C5D7C4084F086049C540D
:108D0000521C92B28C78641E9442EFDC53F8022F0E
:108D100000925A6801929A6802921A4DC0EBC00202
:108D2000497802EB00167419342909D035291CD072
:108D30003729B5D1A85D0028B2D00720A070AFE7D1
:108D4000A85D20B1E11C0C226846FBF70EFB012058
:108D5000A855002161700099C4F803100199C4F866
:108D600007100299C4F80B10E8E7A85D002897D017
:108D70000520A070DFF810C000DF3230C4F8130007
:108D80008EE7000085300020A998000870B5002407
:108D9000224E0125C4EBC40000EB0410315C89B302
:108DA00030448078082828D2DFE800F02D0404043D
:108DB000082D1C126006000E002102E06006000E65
:108DC0000121FEF735FE05EB4400C0B2022112E09E
:108DD0006006000E0021FEF72BFE05EB4400C0B23A
:108DE000062108E06006000E0021FEF721FE05EBDB
:108DF0004400C0B20121FEF71BFE641C14F0FF0406
:108E0000C8D070BDFFE76006000E0021FEF710FE1F
:108E100005EB4400C0B20021EDE7000085300020E2
:108E200070B5094D002400BFC4EBC40000EB041072
:108E300028441721FBF75BFA641C14F0FF04F3D0FD
:108E400002490020487070BD853000208C00002051
:108E5000F0B591B089256B468DF80050DE1C8DF879
:108E60000100D41C2448E4B28DF802408088032716
:108E7000050A8DF803508DF804000525002007E051
:108E800011F800C003F805C06D1C401CEDB2C0B263
:108E90009042F5D3E01C8DF840009DF800008DF85D
:108EA00041009DF801008DF84200002010AA641EC8
:108EB0000EE000BFB0FBF7F107FB110116F800C090
:108EC000515C81EA0C0181F086013154401CC0B232
:108ED000A042EFDB0021084603E01A5C5140401C31
:108EE000C0B2A842F9D359556D1CE9B21846FFF734
:108EF00061F911B0F0BD00008C0000200848006846
:108F0000C0010BD507480068C00707D00548803866
:108F10000068002802DA0449012008707047000048
:108F2000FCED00E0800E00E0F80000204FF0604211
:108F3000D36F002BFCD0436BD367D36F002BFCD0D7
:108F4000C07840EA0120A2F87C0070474FF06041F1
:108F5000CA6F002AFCD081F87C00704770B50546C6
:108F600009484FF480740460084EE9B23046FFF7B8
:108F700067F840213046FEF7CAFF0028F9D00248C2
:108F8000001D0460284670BD1008014000380140F3
:108F900070B5C1B2C0F30725C0F30743000E83EAE2
:108FA000000481EA0502624002F00F0614094A1922
:108FB00018440D4D104400F00F02C0F30313A85DD8
:108FC000AA5C10354840EB5C424082EA03012B5D0D
:108FD0004B401B0603EB014101EB0221084403490E
:108FE000884200D2084470BDB69B0008545C1A0544
:108FF00010B5002100F084FABDE8104000F070BA0E
:10900000FCF794F901210846FEF75EF901211548A5
:10901000FCF702F9FBF736FF134C02212046FCF760
:1090200027F9D8B1002202212046FCF72CF9FCF7E1
:10903000A7F902212046FCF71BF988B10022022182
:109040002046FCF720F9FCF7C9FAFBF781F8074A3C
:1090500007490848DFF820C000DFFEE70122E2E709
:109060000122ECE70002300000080140980D0020CA
:1090700001B00400E95600081597000804490B6880
:1090800004490A88014604A0FFF70CFBFEE7000034
:10909000440000203C0000200D0A5B4F535F4572E6
:1090A000725D6572725F636F64653D256420463D45
:1090B00025642C4C3D256C7500000000FEE7000087
:1090C000074801684FF0E0204161002181610721DC
:1090D00001610448016841F07F4101604017704719
:1090E000389D000820ED00E07047704750E8001FF1
:1090F00031B10B6840E80032002AF7D108467047CA
:10910000BFF32F8FFAE7000070B50D46002812D08C
:109110004FF6FF71084C884204D22268014610467F
:1091200000F01CFA20684570044800F0C3F8BDE860
:10913000704000F0DBBA70BDE4000020D440002095
:109140000F4810B50D4942680E480B6800689342FD
:1091500004D00A60CB88421E1A448A808A8880B272
:1091600082420AD100200860054800F0A3F80146B9
:10917000BDE81040024800F015BA10BD04010020FF
:10918000D4400020F400002070B51A4DE868002893
:109190002ED0A88A401EA882002623E0A06838B1FD
:1091A00061684160606810B1A16881606660A66016
:1091B00010482146183800F0F5F9A08AA882607896
:1091C000042804D10C49E08A09880844A0820120BF
:1091D000607084F82500E068E860E06808B1056127
:1091E000E6602661A88A002802D1EC68002CD5D15F
:1091F00070BD0000EC400020F400002070B50400B9
:109200000FD00D4DA17801262868827891420CD9A3
:1092100000F0E4F9286846702046BDE8704000F090
:1092200065BA064800F046F8F7E766702146BDE8E3
:109230007040024800F0B6B9E4000020D44000209D
:109240000321FFF761BF000010B50446008B0843FF
:1092500020836278618B062A16D0052A17D108422E
:1092600015D001EA0002628388432083204600F083
:10927000BFF901206070022084F825002146BDE876
:109280001040034800F08EB931EA0002ECD010BD66
:10929000D4400020814202D342688A4201D8012092
:1092A000704750E8002F0A6040E80012002AF8D109
:1092B000002070470146406842684A600B780022EF
:1092C000022B05D0012B03D0032B01D04260704745
:1092D00043680BB1996042608260704770B5044684
:1092E00000201546207001226270A17084F82410BD
:1092F0006060A060E06020612062A082E082208344
:10930000608384F8250084F82600208D18B905486C
:10931000FFF7ECFE206329462046BDE8704000F0D0
:109320000FB8000018140020034800210160034911
:109330000988C1807047000004010020349D0008A6
:1093400010B5028D920803D10F4A1288C2F38D0224
:10935000036B03EB8202530700D5121F4FF080739B
:1093600042E9021300231C46B2F1400242F82340B6
:109370005B1C0E2BFAD3C3691362C2624163006B9C
:109380000249016010BD0000309D0008A52E5AE280
:109390002DE9F041044640680F464FF0000804F103
:1093A0000C0620B1617802291DD0A089E8B3A089FC
:1093B000E18988424ED2208904EB8000C0F8107009
:1093C000D6E85F0F401C81B2C6E8501F0028F7D1D5
:1093D0002089401C80B22081E189884201D1A4F813
:1093E0000880BDE8F081406800B10120607020462F
:1093F000FFF760FF80F825802289054604EB820292
:10940000C0694146C2F81000D6E85F0F401C82B226
:10941000C6E8502F0028F7D12089401C80B2208157
:10942000E28990420BD1218109E0FFE72046FFF756
:1094300041FF0546C0690421076085F82510012019
:109440006870284600F0D4F82946BDE8F041044889
:1094500000F0A8B8BDE8F0410320FFF70FBE000000
:10946000D440002070B51B4801210268517000688B
:1094700000F0B4F8184D6C7818E000BF05EBC4019B
:1094800048680278EAB1012A20D000F0E3F8E878D1
:10949000641C844200D100240F48801CD0E84F1F78
:1094A000491EC9B2C0E8421F002AF7D1A878002897
:1094B000E4D16C700948FFF7FDFEBDE8704000F094
:1094C00015B9098989B2FFF7BFFEE0E78968FFF7A0
:1094D0005FFFDCE7E4000020301B0020D4400020C8
:1094E0000548017811B101214170704703494FF0DF
:1094F0008050086070470000EC00002004ED00E0A0
:10950000F0B4154DAB1CEE784FEA0507D3E84F2FAA
:10951000B24202D1BFF32F8F11E0521CD4B2C3E884
:10952000424F002AF2D100BFD7E84F2F541CB4425B
:1095300000D10024E4B2C7E8434F002BF4D1EB780C
:10954000934205D905EBC202C2E90101F0BC7047A4
:10955000F0BC0220FFF792BD301B0020104A10B56E
:10956000D368ABB113469B8A03E08CB12246A48A30
:109570002344D4688B42F8D3C460D0600261C468CD
:1095800004B12061591A8182908A401A908210BDDC
:109590000024C460D060C91A02619182848210BD27
:1095A000EC40002030B502780023022A03D0012AC3
:1095B00001D0032A00D101238C7800E010464268D4
:1095C00012B19578A542F9D24A6041601BB102B14F
:1095D0009160886030BD0020FBE7000003494A68C5
:1095E000426000228260486070470000D440002042
:1095F00010B5016900290ED0C268CA60C368002294
:109600003BB18B8A848A23448B82C3681961C26010
:1096100000E08A82026110BD816839B142684A6007
:109620004168002901D0806888607047054906E0DC
:109630004A68824202D1406848607047114600295A
:10964000F6D17047D440002002220270002242600E
:109650004180704710B5416879B1FFF72BFE044691
:10966000FFF7C6FF01206070032084F82500214623
:10967000BDE810400348FFF795BF4188491C418071
:1096800010BD0000D440002010B50C46418819B12F
:10969000491E4180002010BD34B10A4A4368116858
:1096A00023B1FFF77FFF07E0012010BD4160136881
:1096B000002159601168886007212046FFF724FDCA
:1096C000F2E70000E400002006480068D0E90B1033
:1096D000814203D300680449884202D00120FFF789
:1096E000CDBC7047E4000020A52E5AE207490222B3
:1096F00048604270064A1278002A05D006C98A429C
:1097000002D0C078FFF722BC70470000E4000020C0
:10971000F80000202DE9F047164688468146FFF7FD
:10972000EDFB002004463E4A3E4902E042F820405C
:10973000401C0B889842F9D33B48382201883B48AB
:10974000FEF7FBFF3A48008880B240F000423948FB
:1097500001683948FEF7F1FF384808220188384887
:109760000068FEF7EAFF374FFF25374AFD703C855A
:1097700000213846FFF7B2FD3448042101704460EF
:1097800033480170C46004618482F86A2030FAF7BB
:10979000D9FC304831490760022078702E480470A7
:1097A00044700978C170FFF7BFFD2D48016841F48E
:1097B0007F0101600068290601EA00202849C043B2
:1097C0001439B0FA80F00968C0F10800C1F3022131
:1097D000814200DB481C2249091F0B686FF0807230
:1097E000824063F317020A60FFF76AFC1D490028F4
:1097F00008600DDB00F1E02181F8005400F01F0249
:10980000012191404011800000F1E020C0F80011DA
:10981000324641464846BDE8F047002300F06AB8AA
:10982000341C00202C9D0008489D00084812002090
:10983000309D00084C9D000818140020529D00081F
:10984000500000209C400020BD900008D440002023
:10985000EC400020E4000020301B0020509D000858
:1098600020ED00E0F00000200C4810B50268012156
:1098700051700068FFF7B2FEFFF762FC084801680C
:10988000491C0160FFF780FC00F014F80548FFF761
:1098900011FDBDE81040FFF729BF0000E4000020E3
:1098A000F4000020D4400020014800687047000008
:1098B000F400002070B50D4C2068002815D0A08859
:1098C0000B4E401EA0800AE0E888FFF70EFCA88837
:1098D000A0802868206029463068FFF7DBFCA0885C
:1098E000002802D12568002DEED170BDFC000020BB
:1098F000500000202DE9F0411E46174680460C46D8
:1099000011F0FF0F00D14C1C1948FFF7EFFB0500C9
:109910002BD0200A2F632885E1B242462846EE610B
:10992000FFF7DCFC01241348134905E000EB840237
:1099300052F8042C22B1641C0A889442F6D90024FF
:1099400000EB8400E6B240F8045C0C48EE7000784E
:1099500018B101212846FFF7E9FA2846FFF74EFC27
:109960000748006880F825602046BDE8F0810000C7
:1099700048120020341C00202C9D0008F800002014
:10998000E40000202DE9F05F544DDFF848B1DFF826
:1099900048A129684FF000084FF00509012610B1D1
:1099A000CA7882423FD1474681F80180FAF7CDFB61
:1099B0002968C862FFF788FE2868B046046A18E084
:1099C0006068A8B12046FFF775FC064680F8259030
:1099D000FFF70EFE86F8018031464148FFF7E2FDB1
:1099E000A4F80280A660316AE1603462E46800E0B5
:1099F000E468002CE4D12868C2780AEB820141F8BF
:109A0000047C016B3748FFF745FC286807639BF827
:109A1000001011B10021FFF789FA33482968FFF7D8
:109A200039FC2F6051E03149098888420ED80AEB91
:109A3000800757F8045C4DB12846FFF7EDFD284636
:109A4000FFF7D6FDCA46B1462C6A1BE0FF20BDE8F1
:109A5000F09F6068A8B12046FFF72CFC064680F80E
:109A600025A0FFF7C5FD86F8019031461C48FFF799
:109A700099FDA4F80290A660316AE1603462E4685E
:109A800000E0E468002CE4D147F8048C4446154813
:109A9000296BFFF7FFFB2C639BF8000018B1002136
:109AA0002846FFF743FA29460F48FFF7F3FB0C4817
:109AB00040688278094801688B789A4208D981F811
:109AC000019001680648FFF76DFD0020FFF796FB47
:109AD0000020BCE7F8000020341C0020E400002037
:109AE000D440002018140020481200202C9D0008AB
:109AF000114810B5436801221049002B0ADA4FF0D3
:109B0000E0240523236102700A6803EA92628270EE
:109B100050060FE003F01F0402FA04F45B119B00EF
:109B200003F1E023C3F8804102700A68C2F30072B7
:109B30008270D006086010BDEC00002004ED00E04B
:109B400002480068002800D0C0787047E400002078
:109B500070B5114900200A464B68104C9278002BD2
:109B600009DA4FF0E02507232B6108704B7842EAB1
:109B7000830292060DE003F01F060125B5405B113C
:109B80009B0003F1E023C3F8005108704B781A439F
:109B900012072260487070BDEC00002004ED00E068
:109BA00004E02C2901D1521E04D0401C0178002968
:109BB000F7D10020704712040C0916DC1351ECEEAB
:109BC000553DDC34CE1C526174656C616E2D594874
:109BD0006F6E67323331652B93535EC9A8108CC00A
:109BE00061BE671443751C11BC15D21D98DF4AE293
:109BF0009159E35797DB66D51B4D72C139C248A511
:109C0000D0547C287647EEBDB36F9D71F23CC83FBF
:109C100080A4372256943E0904020A51EB9678B488
:109C200060162487A6D99E2ECD23BBA103060C085F
:109C3000B8F88BD3A71F9545C3F90DE13D20171246
:109C40001A1E7F7974706C683A646231D1E02130F9
:109C5000276A6E6D6B63448A8386BFB9D60ED7F3CD
:109C6000F6FC338840F7C4DA692C2F29B68EB78FFB
:109C70003B9936D8A00789BA8482D4B22618DCE88A
:109C8000EFE985DD8D25B52D2AFBF1018190B10B22
:109C9000FD0558FFF50FC57DCB13C6CC4BCF464C09
:109CA0004FCACE4942C75D5B733432FE5C58F0E761
:109CB000B07A7E4E507755ADAB7BE6ED415FE5FA6D
:109CC000525AEA929AF4359B9CA3ECAC9FAFA93808
:109CD000A2AAAEE4DE192B51495552433A20227212
:109CE000656376222C000000409E00082C9E000830
:109CF000209E0008389E0008309E0008649E0008E0
:109D00005C9E0008F89D0008449E00086C9E0008B8
:109D1000109E0008189E0008009E0008089E00087B
:109D20004C9E0008549E0008749E00080800000025
:109D3000C8000001050001007FFC0A0000000000CF
:109D40001027000005000000CC01000018070000EB
:109D5000200034001640EF001540EF0001471F00BF
:109D60001520C2001640A100000000004B000400B6
:109D7000004040404040404040404141414141401E
:109D800040404040404040404040404040404040D3
:109D90004005020202020202020202020202020262
:109DA0000220202020202020202020020202020267
:109DB00002029090909090901010101010101010BF
:109DC00010101010101010101010101002020202CB
:109DD000020288888888888808080808080808080F
:109DE000080808080808080808080808020202020B
:109DF00040000000719D0008534554494400000094
:109E000052444E414D45000053444E414D450000E3
:109E100052504E414D45000053504E414D450000BB
:109E200044454255474C4F4700000000544700004E
:109E30005253494D000000005353494D00000000AB
:109E4000544D00005250534E000000005241534503
:109E500052000000534153455200000052534552F6
:109E60005645520052564552000000005245424F9E
:109E70004F54000000000000415432354446333254
:109E800031000000464D32355133320057323551E2
:109E9000333200004D5832354C3136303600000038
:109EA0005732355131360000C89E000800000020AE
:109EB000140100001C870008DC9F0008140100202A
:109EC000F44300002C870008000000006400E80351
:109ED000B80B701730750A001E003C00B400680112
:109EE0000000000000000000000000000000000072
:109EF0000000000000000000000000000000000062
:109F00000000000000000000000000000000000051
:109F10006400000000000000541C0020000000004D
:109F20000000000000000000000000000000000031
:109F30000000000000000000000000000000000021
:109F40000000000064000000D007000001010000D4
:109F50000000000000000000000000000000000001
:109F600002040608000000000102030401020304C9
:109F7000060708090000000000A24A0400000000D3
:109F800000000000010203040607080900000000A9
:109F9000000000008C9E0008A09E0008789E00082B
:109FA000949E0008849E0008749E00080000000033
:109FB00000000000000000000000000000000000A1
:109FC0000000000000000000000000000000000091
:0C9FD00000000000000000000000000085
:04000005080041317D
:00000001FF
